:100000005728FF3FFF3FFF3FFF00030E8301A4007F
:100010000408A3000A08A5008A017108A700700857
:10002000A6002108003A031D2E2800308618013052
:10003000F1007108003A031D1F28A00A2028A00320
:100040002008093A031D26280130A0002008003AA4
:10005000031D2C280830A000B52046280030861843
:100060000130F1007108003A031D3828A00A392830
:10007000A0032008053A031D3F280130A0002008F6
:10008000003A031D45280430A000F3208B108F0197
:100090008E010C102708F1002608F00025088A00C0
:1000A00023088400240E8300FF0E7F0E09002130F8
:1000B00003138312900085018601E73083168500C3
:1000C00083128501FF308316860083128601A20108
:1000D0008F018E010C1001300C05F1007108003AFF
:1000E00003197628A20A8F018E010C100530220216
:1000F000031C6B2836309F000F3083168600831256
:100100008601873083168100D0308B000030831247
:10011000851B0130F1007108003A031D9128A101EF
:1001200093280130A1000130A0008F018E010C1036
:1001300003138312003006190130F1007108003AF0
:10014000031DB02801300C05F1007108003A031DB1
:10015000AC2883168615AF28031383168611B3289F
:100160000313831686159828B428D02880300313EB
:1001700083128600F228A0308600F2282030860004
:10018000F22860308600F22840308600F228503095
:100190008600F22810308600F22890308600F2287F
:1001A000031383122008013A0319B6282008023AE3
:1001B0000319BB282008033A0319BE282008043A73
:1001C0000319C1282008053A0319C4282008063A53
:1001D0000319C7282008073A0319CA282008083A33
:1001E0000319CD2808000229A030031383128600CA
:1001F000142960308600142950308600142990306C
:1002000086001429031383122008013A0319F428E5
:100210002008023A0319F9282008033A0319FC2898
:100220002008043A0319FF280800FF3FFF3FFF3F63
:02400E00703F01
:00000001FF
